:030000000219FDE5
:03000B000200A848
:03002B000201646B
:03005B000202EEB0
:030073000202D4B2
:1000800002030406080C10182030406080040608A3
:100090000C10182030406080A0C000070F1F3F05E3
:1000A000050D050305030302C2AFC0D0C0E0206206
:1000B00017E5256002E473E525F4F58A758B00D217
:1000C00062D0E0D0D0D2AF3285268AC262E526F473
:1000D0006036306803207210758B00D0E0D0D0C23B
:1000E00090C291C292D2AF32C290C291C292206E9F
:1000F0000D20660A7401D5E0FDE57EF45290758B03
:1001000000D0E0D0D0D2AF32758A00C28DD2620169
:10011000FE01B7306805206602D29001B73068054D
:10012000206602D29101B7306805206602D29201A2
:10013000B7D29330680A2066077405D5E0FDD290E7
:1001400001B7D29430680A2066077405D5E0FDD265
:100150009101B7D29530680A2066077405D5E0FD95
:10016000D29201B7C2AFC2AD53E6EFC0D0C0E0D269
:10017000D3D2AFC2CEE52A6007207449152A21C523
:100180007800790020742EE580307E01F430E6029C
:1001900078FF53DACF207E0343DA20307E0343DA40
:1001A00010C2D8C271E580307E01F430E60279FFDA
:1001B000C3E89970CB306103752A18207403752A3F
:1001C00018885FD27020740DE52B6004152B21D5A3
:1001D00043DA01C2D82070024137A85F206102C211
:1001E00070207431C3E894F0400374F0F8E8C4540C
:1001F0000F28F87984B703024115C313C31387216D
:10020000200802C313200A06C3C898F8411528F82D
:10021000500374FFF8C3E895685003E568F8882236
:10022000E52D54066011E533C313C31324062522BC
:10023000F52250037522FF852224A824C3E52495C6
:10024000644002A8648825E5697002417BC3E8AA7E
:10025000699A5003E8FAE4F9EAC333FBE56BF45B0F
:1002600029400D256AF8E56A6002156A400B417B5A
:100270000AC3E56A9A5002056A78FF8826C26EC3EF
:10028000E52694F84002D26EC3E52594404002D2A0
:100290006420CF0AD0E0D0D043E610D2AD32C2CF36
:1002A000053A7801E52A6005307402152AC3E55F36
:1002B0009401400575620041CA756300756C00E5E4
:1002C000622401F56250037562FFD0E0D0D043E6AE
:1002D00010D2AD32C2AFC0D053E67FC2607591007C
:1002E000855694855795759104D0D0D2AF32C2AF60
:1002F00053E6EFC2ADC0D0C0E0C0F0D2D3D2AFA8B9
:10030000FBA9FCC2D8307102615553DACF207E03BD
:1003100043DA10307E0343DA20D271E580307E016B
:10032000F420E602612C88278928A18253DACF20A5
:100330007E0343DA20307E0343DA10C2D8C2713024
:100340007402A16E7800E580307E01F430E602A1EF
:100350006E885FA15653DACF207E0343DA20307EC9
:100360000343DA10C271206102812E53DACF207E5E
:100370000343DA10307E0343DA20C2D8D271885AA0
:10038000895BC3E89558F8E99559F97B007E087AAE
:1003900000C3E8948CE994005005755E00812088C4
:1003A0002178A2E6A8216055C3E894C8E9940050DA
:1003B00008E4D2E4FB7A0A61FBC3E89468E994019B
:1003C0005008E4D2E3FB7A0F61FBC3E894D0E994D0
:1003D000025008E4D2E2FB7A1E61FBC3E894A0E974
:1003E00094055008E4D2E1FB7A3C61FBC3E89498A1
:1003F000E994085008E4D2E0FB7A787E00C3E895DF
:100400005CFCE9955DFD30E70AECF42401FCEDF4B9
:100410003400FD755E00C3EC9AED9E5003755E01DD
:10042000885C895D855A58855B597802A156C3E876
:100430009527F8E99528F9307C02A13A307B02A192
:100440003A307A02A1332075028151E9FDE8FC813E
:1004500070E9C313F9E813F8307902A133E9C31343
:10046000F9E813F8307802A133E9C313FDE813FC6F
:0F04700020612CC3EC941CED940240028187EDB7
:10047F00701EC3EC94C850180529E5297002152980
:10048F00C3E529940A5002A16E755F00D270A16E68
:10049F00E529600215297888E6F97400207F08782D
:1004AF0096B90302789EE624FAFEE43400FFC3EC0B
:1004BF009EFCED9FFD9208B90310A208500720760D
:1004CF0009D27681D9307602C276A2085016B903C6
:1004DF000DECF42401FCEDF43400FD0204F378007C
:1004EF007900A13AB90315EC33FCED33FDC3EC945D
:1004FF000AFCED9400FD50047C007D00C3EC94FFDA
:10050F00ED9400400678FF7900A13AEC8575F0A4D0
:10051F00C5F0A2F733F87900400302055678FF794A
:10052F0000020556E9C313F9E813F8307C0EE960B1
:10053F000278FFC3E81338F8E43400F9C3E894FFF6
:10054F00E99400400278FF885FD270206102A16EAB
:10055F00741FF4552F4BF52FC274EB7002D27475C4
:10056F002A18307403752A0A306102A1822074039D
:10057F0053DAFE207403752B06D0F0D0E0D0D0D222
:10058F00AD43E6103279010205B279030205B27963
:10059F000A0205B2791E0205B279640205B279C862
:1005AF000205B27817E4D5E0FDD8FAD9F6227A140D
:1005BF007B780205D97A107B8C0205D97A0D7BB432
:1005CF000205D97A0B7BC80205D97902B27DE4D234
:1005DF0094D5E0FDD291D5E0FDC291D5E0FDC29456
:1005EF00D5E0FDD290E576D5E0FDC2907496D5E0CA
:1005FF00FDD9D9EAF8D5E0FDD8FBDBCED29422C3E2
:10060F007C007D0075F00005F0EA33FAEB33FB5008
:10061F00F6EB13FBEA13FAC3E9FFE8FEE89AF8E9F1
:10062F009BF95004EFF9EEF8B3EC33FCED33FDD545
:10063F00F0DFEDF9ECF822E889F08A20D2D4F8A99E
:10064F00F07B0030F70B7BFFF42401F8E9F4340062
:10065F00F9E88520F0A4ADF0F8E98520F0A4AFF01B
:10066F00FEED2EF974003FFA7C04C3EA13FAE91386
:10067F00F9E813F8DCF48BF030F70AE8F42401F80A
:10068F00E9F43400F9E889F0C2D4F8A9F02222C3C2
:10069F00E54113F9E54013F8C3E54598F8E54699A8
:1006AF00F9500CC3E89480E994FF40160206D5C3B5
:1006BF00E8947FE9940050030206D5787F79000211
:1006CF0006D5788079FF884A894B22E54A2547F875
:1006DF00E54B3548F9854B20E4300701F43549FAED
:1006EF0030E709C3EA94F04015020713C3EA940FE9
:1006FF00500302071378FF79FF7A0F020713780070
:10070F0079007AF0C3E5249564500AC374019524E7
:10071F00500B020731E54B20E70E020731E54B3056
:10072F00E706884789488A492278A4E6FAC3E54A4A
:10073F0033F8E54B33F9D146E930E70BC3E8948042
:10074F00E994FF4013E16BC3E8947FE994005002F2
:10075F00E16B787F7900E16B788079FFE820E7150E
:10076F00C3E52398F84009C3E894014003020792B8
:10077F007801020792E8F424012523F840030207C9
:10078F009278FF884C2278A5E6FAA848A949D14665
:10079F00E930E70CC3E89401E994FF40160207C65D
:1007AF00C3E894FFE9940050030207C678FF79006D
:1007BF000207C6780179FFE920E715C3E54C98F8E1
:1007CF004009C3E8940140030207ED78010207EDE9
:1007DF00E8F42401254CF840030207ED78FF882444
:1007EF002278FFC26420693D206A12D264C3E541BA
:1007FF00940A4009C3E52594405002C26479A1E7E9
:10080F006023E541601F74FF8541F0848539F03026
:10081F006A0375F005A4F8C5F0600278FFC3E89588
:10082F00675002A867886622C3E5409440E541946B
:10083F0001E5665003140148046002F566220208C0
:10084F00502275E890227883E6FFE5E820ECF7A8C0
:10085F00BDA9BE0573C3E57394084052757300E9D3
:0D086F00FA79A0E76044EA7007E574601BA9
:10087C0002088BC3E895746010E5745006600C1484
:10088C000208970460F9020897E574F574C394F6AE
:10089C00401B7564C0C394064013756480C39406F2
:1008AC00400B756440C39406400375640075BB0E21
:1008BC0022E564F460020564E573B4070375BB10AC
:1008CC0022743279A687F0A4C5F0A2F733F8C3E8F6
:1008DC0095644002A8648822882488258826886725
:1008EC00227540007541F022C2AF75C820A8CCA972
:1008FC00CDAA3A30CF010A75C824D2AFAB3BAC3C81
:10090C00883B893CC3E89BF8E99C206908F930676F
:10091C000241092166AD3D8A3DF9EA9DFA600478F1
:10092C00FF79FFAE3EAF3F8B3E8C3FC3EC9FFCC3C9
:10093C00E99CF542A83BA93CC3E89EF8E99FF9C3A2
:10094C00E54113FBE54013FAE82AF540E93BF54194
:10095C0050067540FF7541FF21B0AA40AB41AC4039
:10096C00AD417E047F02C3EB940440021E1FC3EB17
:10097C00940840021E1FC3ED13FDEC13FCDEF7C3FD
:10098C00EA9CFAEB9DFBEF6009C3E913F9E813F855
:10099C00DFF7EA28FAEB39FB8A408B4150067BFFE4
:1009AC008B408B41C3EB94025002D2673069047FB9
:1009BC000321DB7892E6FFC3E537948240110FC325
:1009CC00E53794A040010FC3EF940640027F057EEB
:1009DC0004E541C4540FF9E541C454F0F8E540C4B2
:1009EC00540F28F8C3E89EFAE99400FB4009C3EAC7
:1009FC009402EB940050047A02E4FB4155AA40ABFC
:100A0C0041EBC4FEEAC4540F4EFCC3EA9CFAEB94CF
:100A1C0000FBC3E813C313F8EA28FAEB3400FB8A93
:100A2C00408B41C3EB94024002C2677804EBC4FED6
:100A3C007B00EAC4540F4EFAC3EA98FA4005C394FB
:100A4C000250027A027892E6FF30600241558552DC
:100A5C0056855357D26043E680C3E49AF8E49BF979
:100A6C0030670241EFE8FAE9FBD3E913FDE813FC28
:100A7C0088528953C3EF94036038EF20E00DE82CC3
:100A8C00F8E93DF9ECFAEDFB020AAAE828F8E93995
:100A9C00F9C3E82402F8E93400F97AFE7BFFC3EFCE
:100AAC009403400E8A548B55884E894F8C508D512F
:100ABC006123885489558A4E8B4F8C508D513069E7
:100ACC0020C3E53394034019E542A2E713F8E5553A
:100ADC00F4240138400B20E7087554FFF42401F589
:100AEC00556123E8FAD3E813FC8852C3EF940360F2
:100AFC0020EF20E007E82CF8ECFA610FE82824023C
:100B0C00F87AFEC3EF940340088A54884E8C5061E7
:100B1C002388548A4E8C50E56BC3335002646BF5BA
:100B2C006B306002612D753402D26043E680E52D96
:100B3C0054066026A840A941C3E913F9E813F8C28A
:100B4C00AF53E67F759100C3E498F594E499F5955D
:100B5C00759104D26043E680D2AF22D26575440011
:100B6C00752000306B03752040020B86D2657544EE
:100B7C0000752040306B03752000D2AF78012067E0
:100B8C0022E52D54066002C265C3E541940540136D
:100B9C007802940540087803940540027806306981
:100BAC0002780A206019E544601530690AC3E53300
:100BBC0094034003D53406D2AFD26C81587135D230
:100BCC00AF0000C2AF206726E541C3FB940F400283
:100BDC007B0FEB240530730123306A0274282062EA
:100BEC000123F93069027982E58BC39940B505443C
:100BFC00E59BF45440B52002814230690A08C3E8F1
:100C0C00940A40010861AF2065026186C26553E613
:100C1C007F7591003067107594007595FE75910481
:100C2C00D26043E6806186AE40AF41C3E49EF5944A
:100C3C00E49FF5958129C3E5339402500261863017
:100C4C0065026186D802815661AFC26C53E67F752E
:100C5C009100855494855595759104854E56854F14
:0E0C6C0057D26043E680D2AFE52D54066008F3
:100C7A00206A020533020C92306C0D206B0A206543
:100C8A00071581158102150F227800306405306539
:100C9A00027801E53775F007A4F9E5F028F5F0E9DF
:100CAA00A2F013A2F113A2F213F537C394785003FA
:100CBA00753778C3E53795384008D266C290C29135
:100CCA00C29230600281CC855056855157D260431A
:100CDA00E68022207D11C2AF754302D294C293D21C
:100CEA00AF759F11020EACC2AF754302D294C29582
:100CFA00D2AF759F11020EAC307243207D20C2AF75
:100D0A00754303900142757E10C292D295306204F7
:100D1A00D291A120C294D2AF759F01020EACC2AF8C
:100D2A00754303900142757E10C290D293306204DB
:100D3A00D291A140C294D2AF759F21020EAC207D00
:100D4A0017C2AF75430390011DC292306202D2915D
:100D5A00D2AF759F01020EACC2AF75430390011D5D
:100D6A00C290306202D291D2AF759F21020EAC209E
:100D7A007D11C2AF754304D293C295D2AF759F213C
:100D8A00020EACC2AF754304D295C293D2AF759F1F
:100D9A0001020EAC307243207D20C2AF754305902C
:100DAA000131757E08C291D294306204D290A1BCFE
:100DBA00C293D2AF759F11020EACC2AF75430590B4
:100DCA000153757E20C291D294306204D292A1DC82
:100DDA00C295D2AF759F11020EAC207D17C2AF75B6
:100DEA004305900113C291306202D290D2AF759F2F
:100DFA0011020EACC2AF754305900127C291306251
:100E0A00EBD292D2AF759F11020EAC207D11C2AF08
:100E1A00754306D295C294D2AF759F01020EACC239
:100E2A00AF754306D293C294D2AF759F21020EAC1E
:100E3A00307242207D20C2AF754301900153757E06
:100E4A0020C290D293306204D292C158C295D2AFD6
:100E5A00759F21020EACC2AF754301900131757EB8
:100E6A0008C292D295306204D290C178C293D2AFAE
:100E7A00759F01C1AC207D16C2AF75430190012751
:100E8A00C290306202D292D2AF759F21C1ACC2AF7A
:100E9A00754301900113C292306202D290D2AF75AB
:100EAA009F01C26622900111757E00C290C291C252
:100EBA0092D293D294D295C26222788076FF087633
:100ECA00FF0876FF0876FF08760308760408760B93
:100EDA00087603087601087601788C76010876FF91
:100EEA000876FF0876FF0876FF0876FF087603087B
:100EFA0076FF0876FF0876FF0876250876D008760A
:100F0A00FA0876FA0876040876FF08760108760069
:100F1A0008767A0876FF08760108760108760008CE
:100F2A007603227887E6FFC272BF0302D2727888FC
:100F3A00E6C394036008C27DE630E102D27DC27E38
:100F4A007889E630E102D27EC3EF94026008758E9A
:100F5A0001D273020F65758E00C273227880E6147F
:100F6A009000809378A4F67881E6149000809378B4
:100F7A00A5F67886E61490008D9378A6F6789CE616
:100F8A007538FF75390CB402067538A075390AB47C
:100F9A00030675388275390578A3E61490009A938A
:100FAA00F569D1AF22227896E6FA7897E6FB788837
:100FBA00E6B40305C3EB940EFB307F047A007BFF93
:100FCA00C3EB9AFCC3948250027C82757500057546
:100FDA00EC8575F0A4C3E5F0947D40F222D27FF14E
:100FEA00B01205A37A007B007C10120599E55F2AEE
:100FFA00FA74003BFBDCF37C04C3EB13FBEA13FA41
:10100A00DCF7FEC27F120FB022E5EF20E60375205F
:10101A00000520903FFFE520146006901DFF146034
:10102A00009304600375EF1053D9BF7581C043FF65
:10103A008012059475EF0043B203E5B3240420E758
:10104A000DF521E5E320E0068521B343E301120E05
:10105A00AF7580FF75A40075F1D075D4BF7590780F
:0F106A0075A53F75F2BF75D54075A60175E241BA
:10107900E4F8F6D8FD756B01120EC4121551789873
:101089008676753001C2AF1205AD1205BD1205A3F2
:101099001205C41205A31205CB1205A312166A1272
:1010A90005AD1205AD1205A8C2AF78FA79FA3086F6
:1010B90007D9FBD8F7021C00120F2D120F66120F69
:1010C900AF120FB078988676120EAF758850758971
:1010D9001275C82475910475D84075A82275B8028F
:1010E90075E690759B80759D0075D10775BC58751F
:1010F900BB0E75BA1175E880120594D2AF12084D6E
:1011090053DACF207E0343DA20307E0343DA1043DB
:10111900DA01C2D8C2711205ADD2617B037A0CE53E
:101129005E70077A0CDB030210B11205A32070036D
:101139000210B1C270E55FC3940240E1E52F541F6C
:10114900856160F561B560D5DAD5C26153DACF2022
:101159007E0343DA20307E0343DA10C2D8C27178A5
:10116900A2E67008D274E52F54E0F52FC2757529EF
:10117900001205A8307409C3E529940A4002D27502
:1011890012059978023074027800C3E55F9840F03F
:10119900C2AF1205BD1205BD1205BDD2AF1205AD14
:1011A900754D007888E6B403024191120599788C4F
:1011B900E6C394015003021291E530C39401500330
:1011C900021291207435C3E55F94FF500302129116
:1011D900C2AF1205D2D2AF1205A8C3E55F94015080
:1011E900EFC2AF1205BD12059E1205BDD2AF1205A1
:1011F900A8C3E55F94FF40E90216EF7F05D27F128D
:101209000FB01205A8C2AFC27F120FB0AE5FC3E51F
:101219005F947FD2AF407B120594C2AF1205D2D240
:10122900AFDFDA120FE7C3EE94057897F61205AD32
:101239001215931216727F0AD27F120FB01205A8E7
:10124900C2AFC27F120FB0AE5FC3E55F947FD2AF6A
:1012590050E4120594C2AF1205BD12059E1205BDD8
:10126900D2AFDFD4120FE7EE24057896F61205AD5A
:101279001215931216A11205A8120FB0C3E55F94B7
:10128900FF500221CC0216EFC3E55F954D4003855F
:101299005F4D1205A878017988E7B403027805C380
:1012A900E55F98400221ACC2AF1205D21205D212F5
:1012B90005D2D2AF1205AD753000E4F531F532052E
:1012C90031E531F470390532789AE67819146012EB
:1012D900783214600D787D14600878FA146003750B
:1012E9003200C3E53298401715327531B4789986C2
:1012F90076C2AF1205D2D2AF789886761205A812B7
:10130900059EE52A700530740201B1780120740246
:101319007806C3E55F9840A77888E6C3940360031D
:101329001205A8E52A70030210B1C2AF120EAFE48C
:10133900F522F523F524F525F526F56AD2AF78854A
:10134900E6C333F568E4F545F546F547F548F5494B
:10135900F573F52CF52DF53775730875BB10120566
:1013690094120851E5E820ECFBA8BDA9BEE970017B
:10137900F8887412085575730875BB107887E6FEEE
:101389007602120F2D7887EEF6C2AF7564FF120848
:10139900CD852264852265852266D2AF75220175C5
:1013A900240175250175260185636C756D017888A1
:1013B900E6B40307C27D307602D27DD268D2697560
:1013C9003300120E15120E3A1208ED1208F4120823
:1013D900ED1208F41208ED0213F0C2AF120F2DD26C
:1013E900AF75730075BB0E120B7812069D120C9324
:1013F900120CDD1208F4120B67306D0312069E20E1
:1014090067031207F0306703120837120C93120DA5
:10141900021208F4120B78306D031206DA120C93DB
:10142900120D791208F4120B67306D031207381286
:101439000C93120D9E1208F4120B78306D031207EB
:1014490095120C93120E151208F4120851120B671B
:10145900120C93120E3A1208551208F43069322010
:0E1469006B2F85676485676585636C756D0103
:1014770079187A0CC3E53399400CC269D26A8A3568
:101487007564FF02149AC3E55F940140030213F0E9
:10149700021517306A1B206B18E535147004C26AF1
:1014A70061E3F535C3E55F940140030213F00215CC
:1014B70017753600C3E5627882985054307404E596
:1014C7002A604D7888E6B40317207D0520760781CA
:1014D700E730760281E7206B07D26B856764812F3F
:1014E70078F0306B058567647820C3E54198500232
:1014F70061F0306B1BC26BC27D307602D27DD26A3F
:1015070075351285676461F00536E55F6002A11ADB
:10151700753600C2AF120EAF7887E6FE7602120F5D
:101527002D7887EEF6E4F522F523F524F525F52643
:10153700F568C268D2AF120594120EAF307409C3B2
:10154700E5369405400201B141C3901A0D78201287
:1015570015D5E520B45A0CA31215D5E520B4A5037B
:10156700021573120EC4121593021592901A03787E
:10157700807B0A1215D5A308DBF9901A0F788C7BAC
:10158700181215D5A308DBF9901A2722C2AF121635
:10159700141215EE901A00740E1215DAA3740412C1
:1015A70015DAA374141215DA901A0378807B0A12DD
:1015B70015D9A308DBF9901A0F788C7B181215D967
:1015C700A308DBF9121627121605901A2722E493AF
:1015D700F622E6438F01538FFD75EF0275B7A575A8
:1015E700B7F1F0538FFE22438F02438F0175EF024D
:1015F70075B7A575B7F1901A0DF0538FFC22901AA5
:101607000D745AB1DA901A0E74A5B1DA227A3079CC
:10161700D07820901A40B1D5E520F709A3DAF72250
:101627007A3079D0901A40E7B1DA09A3DAF922AB18
:1016370077A878BB01027984BB02027985BB0302D4
:101647007986BB04027992BB05027987BB060279CA
:10165700A3BB0702799CBB08027988BB0902798979
:10166700E8F7227C051205ADDCFB22C2AF1205BDEF
:101677001205C41205CB1205D212059E1205BD1222
:1016870005C41205CB1205D212059E1205BD12051F
:10169700C41205CB1205D2D2AF22C2AF1205D212A5
:1016A70005CB1205C41205BD12059E1205D21205FF
:1016B700CB1205C41205BD12059E1205D21205CB29
:1016C7001205C41205BDD2AF22AE77AF78C2AF12F2
:1016D70005BD1205BD1205BD12059EDEF21205D22B
:1016E70012059EDFF8D2AF22D172D16AD16A75771F
:1016F70001757801757900D1D07C05AD5F1205AD14
:10170700C3ED955F70F5C3E55F9401400AC3E55FDC
:1017170094FF403202172BD136B193D172C2AF7505
:10172700EF10D16ADCD50579C3E5799403500280BF
:10173700C6D16A0578E5771490009F93F808C3E54A
:101747007898500280AED16AD16A0577C3E577945D
:101757000A5002809C120EC4B193C2AF75EF10D12C
:011767006A17
:0319FD00021013C2
:101A00000E0414FFFFFFFF03040B0301015AA5019D
:101A1000FFFFFFFFFF03FFFFFF25D0FAFA04FF01DE
:081A2000007AFF01010003FF41
:101A40002353757065726D6963726F33703541230E
:101A500023424C48454C4923463333302320202031
:101A60002020202020202020202020202020202076
:101C0000C2AFC2D353D9BF7581C043B20343FF8073
:101C1000752438752503B1C975EF0275E24043F1AB
:101C20004053A4BF75D400D2867DFA780379E67C50
:101C300010752200752300901DD67B0675249875BB
:101C400025013086028142208608D8FBD9F9DCF7CD
:101C500081B4308608D8FBD9F9DCF781B4B189E4C6
:101C600093A3C39A6004DDC381B4DBDBB17B600264
:101C7000812B7B08E493FAA3B15CDBF87A30B15C8A
:101C8000752200752300B17BEAFCEBFDC3ED94FEE9
:101C9000400EB17B8A278B28ED30E0048A828B834B
:101CA000B17B7AC270D8C3ED94FE601350CEBD00F4
:101CB00025EC60097520007521FF0200008100A855
:101CC00027A9280809D804D90281D3B17FEA89AAB3
:101CD000F281C50D81A0C3ED94035049EDA2E092BD
:101CE000007AC5C3E5829400E583941C50902000DF
:101CF00010438F02438F0175B7A575B7F1F030001F
:101D00001FA827A9280809438F01538FFDD804D99C
:101D100002A12089AAE275B7A575B7F1F0A3A10DBC
:101D2000538FFC817C7AC1BD030CE493A3FAB140CC
:101D3000DCF8B138817C817EAA22AB23B15CEBFA5E
:101D4000EA6222752608C3E52313F523E52213F57D
:101D50002250066323A0632201D526EAB1C9B1C986
:101D600075260AEAF4200102D286300102C286B149
:101D7000C9C3134002C201D526EB22B17FEAFB2082
:101D80008602A17F308602A184752608AE24AF2585
:101D9000C3EF13FFEE13FEB1CDB1C9C3EA13308612
:101DA000024480FA30E703632201C3E52313F523DD
:101DB000E52213F52250066323A0632201D526D91C
:101DC000E52265236523F52222AE24AF250E0FDE22
:101DD000FEDFFCD20122424C48656C693437316326
:041DE000F3300601D5
:00000001FF
